:020000040000FA
:10000000102882073F3406345B344F3466346D3435
:100010007D3407347F346F34403479347134733431
:10002000850186018701A501831606309F003F30B8
:1000300085008601870183120A30012087000A307B
:10004000A2008717F4218713F421851C2C28051C96
:100050002C28A20B212836280D30012087002514DA
:100060001522F421051C3128851C3128051A462843
:100070000B30012087001522F4211522F4211522CE
:100080000615051E4128EC21EC2106110130012046
:1000900087001522F421051C4A28051C5228851CBE
:1000A000E9284D280230012087001522F421051C83
:1000B0005628051C5E28851CEF285928033001208E
:1000C00087001522F421051C6228051C6A28851C5E
:1000D000FC2865280430012087001522F421051C26
:1000E0006E28051C7628851C0929712805300120F9
:1000F00087001522F421051C7A28051C8228851CFE
:1001000016297D280630012087001522F421051CC0
:100110008628051C8E28851C23298928013001206A
:10012000870087171522F421051C9328051C9B289E
:10013000851C39299628023001208700871715224F
:10014000F421051CA028051CA828851C3F29A328EC
:1001500003300120870087171522F421051CAD28E4
:10016000051CB528851C4D29B028043001208700C6
:1001700087171522F421051CBA28051CC228851CE6
:100180005B29BD2805300120870087171522F4213F
:10019000051CC728051CCF28851C6929CA280630DC
:1001A0000120870087171522F421051CD428051C7F
:1001B000DC28851C7729D72807300120870087177E
:1001C0001522F421051CE128051C4628851C8529DB
:1001D000E42815229C219D210630A821B421152256
:1001E000023001208700251CF7288518EF289C2164
:1001F0009D210630A821B42115220330012087005B
:10020000251C04298518FC289C219D210630A82145
:10021000B4211522043001208700251C11298518DE
:1002200009299C219D213330A821B42115220530B4
:1002300001208700251C1E29851816299C219D2137
:100240001830A821B4211522063001208700251C72
:100250002B2985182329BB210C300120870003227C
:10026000051830290A3001208700F421051C3529A2
:10027000462815229C219D210630A821B421152253
:100280000230012087008717251C482985183F293F
:100290009C219D211530A821B42115220330012075
:1002A00087008717251C562985184D299C219D21DB
:1002B0001530A821B42115220430012087008717AA
:1002C000251C642985185B299C219D213330A82198
:1002D000B42115220530012087008717251C7229BB
:1002E000851869299C219D211530A821B42115224A
:1002F0000630012087008717251C8029851877295B
:100300009C219D215A30A821B421152207300120BB
:1003100087008717251C8E2985188529BB210C305D
:10032000012087000322051893290A300120870045
:10033000F421051C98298E28080086150519A32983
:10034000851EA6299D29051EA6299D29861108001E
:10035000A30086160708A400D92186122408870066
:10036000EC21A30BA92908000615051EB529EC21CF
:10037000EC210611080085190800051AC529061583
:10038000051EC029EC21EC21061106170615EC21EB
:10039000EC21EC21EC21EC21EC210430A30006152A
:1003A000EC210611EC21EC21EC21A30BCF29061343
:1003B00008000A30A200DF21A20BDB290800203050
:1003C0008700F42101308700F42102308700F421F6
:1003D00040308700F42108002830EF290430A200C3
:1003E000F421A20BF0290800FA30A1006E30A00021
:1003F000000000000000000000000000A00BF82931
:10040000A10BF62908000730A3001522A30B052A2B
:10041000F4210730A3001522A30B0B2AF421073087
:10042000A3001522A30B112A08004B30A100861748
:100430001E2286131E22A10B172A08003730A000A7
:10044000000000000000000000000000A00B202AB7
:020450000800A2
:00000001FF
